:0200000480007A
:100000006F004005732F2034930F8000630AFF03B5
:10001000930F90006306FF03930FB0006302FF038A
:10002000170F0000130F0F2963040F0067000F0064
:10003000732F203463540F006F00400093E19153FD
:10004000171F000023203FFC171F0000232E0FFA6C
:100050006FF01FFF930000001301000093010000E8
:10006000130200009302000013030000930300003A
:100070001304000093040000130500009305000022
:10008000130600009306000013070000930700000A
:1000900013080000930800001309000093090000F2
:1000A000130A0000930A0000130B0000930B0000DA
:1000B000130C0000930C0000130D0000930D0000C2
:1000C000130E0000930E0000130F0000930F0000AA
:1000D000732540F16310050097020000938202012E
:1000E000739052307350447497020000938202015F
:1000F00073905230735000189702000093820202EE
:1001000073905230B70200809382F2FF7390023BEB
:100110009302F0017390023A73504030970200004E
:1001200093824201739052307350203073503030BC
:100130009301000097020000938202ED7390523009
:10014000130510001315F501634C05000F00F00FA7
:10015000930110009308D005130500007300000000
:1001600093020000638A020073905210B7B200003D
:100170009382921073902230735000303725000024
:100180001305058073200530970200009382420119
:1001900073901234732540F17300203093012000D6
:1001A00097200000938000E63751341213018167D5
:1001B000970700009387470123A0200003A70000B2
:1001C0006F00800013070100B753341293838367D5
:1001D0006318770A9301300097200000938080E233
:1001E00037E1BC9A130101EF97070000938747019D
:1001F000A3A0200003A710006F00800013070100D8
:10020000B7E3BC9A938303EF631C77069301400026
:1002100097200000938000DF37C1ADDE1301F1EEBF
:10022000970700009387470123A1200003A7200020
:100230006F00800013070100B7C3ADDE9383F3EEB8
:10024000631077049301500097200000938080DBB7
:100250003701EDFE13011101970700009387470155
:10026000A3A1200003A730006F0080001307010046
:10027000B703EDFE9383130163147700631030021C
:100280000F00F00F638001009391110093E11100C2
:100290009308D00513850100730000000F00F00FD4
:1002A000930110009308D0051305000073000000AF
:1002B0009302600073232034E39462FC739017343C
:1002C00073002030731000C0000000000000000028
:1002D000000000000000000000000000000000001E
:1002E000000000000000000000000000000000000E
:1002F00000000000000000000000000000000000FE
:1010000000000000000000000000000000000000E0
:1010100000000000000000000000000000000000D0
:1010200000000000000000000000000000000000C0
:1010300000000000000000000000000000000000B0
:081040000000000000000000A8
:1020000000000000000000000000000000000000D0
:040000058000000077
:00000001FF
